:10000000C201A029FF3FFF3F0800A800F839A00067
:10001000A00CA00C200C84071121A80000050800EA
:100020002808031C03010006280580069B29A70059
:1000300006108611861183160610861186110F3060
:10004000860583122708C21843283A30A100983049
:1000500031213330A60057201330A10088303121E0
:100060005720643030215720643030212230A600E0
:100070005720283042200C30422006304220C21443
:10008000270843284214A600421C51288611033C2D
:10009000031C562856200730A100D030312103140C
:1000A00008004214FE3C03199B298615421C42108D
:1000B00006140F3086052608F03986040610A60EB1
:1000C0004218572832303021031408002C08A000B1
:1000D0002D08A1000130A200A30164009420031C9C
:1000E0008128A20B6D28FF30A30703186D28A007F5
:1000F000031CA107031C9B29FA30A2000030A300B7
:100100006D280121A8010830A300022194200318C2
:10011000A80AAB1EA801A20CA30B8528AB1AA21338
:1001200002210314220808004608840044088417AA
:100130008004841300052B1B4406FF3E0800A40026
:100140002908031403199B299621031C0800A00009
:100150002518831724088400200880008313A40A2C
:10016000A903A028A4002908031403199B29962198
:10017000031C0800A0002518831724088400200809
:1001800080002E020319C8288313A40AA903B328E8
:100190008001840AA90BC82803149B29A6004608DD
:1001A00084008030C3050830A70003100318C30A79
:1001B000E720A60CA70BD6280000AB1A430CE720BB
:1001C0009E210314E7202F08A3002E08242984135E
:1001D000AB1FF628000844042B1F44068000841738
:1001E00000084404031C440680000229000844045B
:1001F000031C44062B1B4406800084174409800519
:10020000022943172B081F39003EA1002A080E3E81
:100210000318A10A431F31294313A00002304321D0
:10022000312901308A002808073982070134023455
:1002300004340834103420344034803483169B0056
:100240001C141A089B29A301A200FF30A207031C5B
:10025000A307031C9B290330A100E6303121252987
:10026000A101FC3EA000A109031C3C29FF300000B5
:10027000A00703183729A0076400A10F362908003A
:100280000310A10CA00CFF3E0318402920089B2955
:10029000A101A301A20003304D29A80023082102D7
:1002A000031D5429220820020430031801300319C9
:1002B00002302805031DFF309B290038031DFF3045
:1002C0000405031DFF309B29A501A4011030A600E1
:1002D000210DA40DA50D2208A4022308031C230F41
:1002E000A50203187A292208A40723080318230F5C
:1002F000A5070310A00DA10DA60B682920089B29B6
:100300001030A800A101A001A70CA60C031C8E2987
:100310002208A00723080318230FA107A10CA00C93
:10032000A50CA40CA80B842924089B29840031085F
:100330008A003008820083130313831264000800CC
:1003400007309F00831685010516860186148312E7
:10035000FE308A01172001308A0117200615831606
:100360000611573081008312A0308B008B178A1141
:10037000BD298B1B08008A15A72E8A01B9218B1273
:100380008A01B92183164130DE0083128A01B92126
:100390008A15AA248A01B92164008A11051ADA296A
:1003A0008A01B92183162530DE0083128A01B92122
:1003B0008A11E2298A01B92183162930DE008312CD
:1003C0008A01B9218A01B9218A15AA248A01B92191
:1003D00083160430DC0083128A01B9218A15C925ED
:1003E0008A01B9214E30C8008A01B9214130C900C3
:1003F0008A01B9215630CA008A01B9214930CB009F
:100400008A01B9215430CC008A01B9215230CD0083
:100410008A01B9214130CE008A01B9212030CF00B4
:100420008A01B9214430D0008A01B9214930D10074
:100430008A01B9215330D2008A01B9215030D3004A
:100440008A01B9214C30D4008A01B9214130D5004C
:100450008A01B9215930D6008A01B9212030D7004C
:100460008A01B9215630D8008A01B9213030D9002B
:100470008A01B9212E30DA008A01B9213030DB003F
:100480008A01B9213030DC008A01B9213230DD0027
:100490008A01B9214330DE008A01B9215130DF00E1
:1004A0008A01B9218A11DD238A01B9218A15E9243B
:1004B0008A01B9210330A300E8308A0124218A018E
:1004C000B92183160F30ED0083128A01B9218316FA
:1004D0000330DC0083128A01B9218B168A01B9210D
:1004E0008B128A01B92164008A11831683106C1C57
:1004F000831483128318882A8A01B9218316ED0A8E
:1005000083128A01B92183166C1083128A01B921E2
:100510008A01B92164001A3083166D028A11831290
:10052000031CA32A8A01B9218316ED0183128A01D3
:10053000B92183161230DE0083128A01B9218A158F
:10054000AA248A01B9218A01B9218A11AB228A0120
:10055000B9218A016B2A8A01B9210630C60002300E
:10056000C4005430AA00AB01FF30AC00AD0106302E
:10057000A9006630B000B101A50148308A019F2072
:100580008A11031CDA2B8A01B9210630C600023019
:10059000C4005430AA00AB016430AC00AD018A0144
:1005A00066208A11031CDA2B243C8A11031DCF2AF2
:1005B0008A01B92183160130DE00831264000F30F6
:1005C00083165E028A1183120318032B8A01B92154
:1005D0000630C6000230C4005430AA00AB016430BB
:1005E000AC00AD018A0166208A11031CDA2B2C3C79
:1005F0008A11031DF22A8A01B9218316DE0A8A11A3
:100600008312031DDE2A8A01B9210630C60002309A
:10061000C4005430AA00AB016430AC00AD0114300A
:10062000A9002C30AE006630B000B101A501BE308B
:100630008A01B2208A11031CDA2B8A01B9218316A0
:10064000DF0183128A01B9218316DE01831264005F
:10065000143083165E028A1183120318512B8A010B
:10066000B92183165E08673E840000088312B20039
:1006700083165E08BE3E840000088312B400640046
:10068000320834028A110319492B83160130DF0026
:1006900083128A01B9218316DE0A8A118312031D8F
:1006A000272B8A01B921640083165F08003C8A1158
:1006B0008312031D612B8A01B9218A11DA2B8A0169
:1006C000B9218A01B9218316DE0183126400143036
:1006D00083165E028A1183120318862B8A01B921C0
:1006E00083165E08BE3E840000088312B2008316A3
:1006F0005E08673E84008312320880008A01B921B7
:100700008316DE0A8A118312031D662B8A01B92122
:100710003E30CE008A01B92183160730DF008312F4
:100720008A01B9218316DE01831264001430831616
:100730005E028A1183120318BA2B8A01B92183162B
:100740005E08BE3E840000088312B20083165F0874
:10075000483E84008312320880008A01B921831642
:10076000DF0A83128A01B9218316DE0A8A118312F5
:10077000031D952B8A01B921FE308A011720013013
:100780008A0117208A01B92183161230DE008312F4
:100790008A01B9218A15AA248A01B9218A11DD2387
:1007A0008A01B9218A15E9248A01B92183161930F1
:1007B000ED0083128A01B92108008A01B92183164C
:1007C000DE01831264001E3083165E028A118312DA
:1007D0000318042C8A01B92183165E08BE3E8400EA
:1007E000FF30800083128A01B92183165E08A03E83
:1007F0008400FF30800083128A01B9218316DE0A4B
:100800008A118312031DE22B8A01B9218316E401A8
:1008100083128A01B9218316E20183128A01B92168
:100820008316DE01831264001E3083165E028A1571
:1008300083120318A72C8A01B92183165E08483E4B
:1008400084000008DF0083128A01B9210130831679
:100850005E078312B200B301B30D3208483E840034
:1008600083160008E00083128A01B9216400831610
:100870005F08003C8A15831203199F2C8A01B92155
:1008800083165F08E30083128A01B9216400803077
:1008900083165F028A1183120318582C8A01B9212A
:1008A0008A11DC258A01B9218A1577288A01B921A4
:1008B0008A01B92183165F088312A00081308A0162
:1008C0004821B2009F30A00083165F0883128A017E
:1008D0004821B4003208840034088A015D218A115D
:1008E000031D942C8A01B92183165F088312A0008E
:1008F000E0308A014821B200EF30A00083165F0883
:1009000083128A014821B4003208840034088A0125
:100910005D218A11031D942C8A01B9218A11F027C7
:100920008A01B9218A11442D8A01B92183166008F0
:100930008312A00040308A014821B2007E30A0001E
:100940008316600883128A014821B40032088400AB
:1009500034088A015D218A11031DCC2C8A01B9213A
:10096000831660088312A00080308A014821B200FB
:10097000FC30A0008316600883128A014821B4006D
:100980003208840034088A015D218A11031DCC2CB1
:100990008A01B9218A11CA2D8A01B9218316A5308D
:1009A000E30083128A01B9218A1588268A01B921B8
:1009B0006400E03083165F028A118312031CE42C6A
:1009C00040308316DF0283128A01B921640080302F
:1009D000831660028A118312031CF12C8316E00334
:1009E00083128A01B92164009E30831660028A1145
:1009F0008312031C1C2D8A01B921903083165F07D6
:100A00008312B200FF300318013EB3003208A60083
:100A10003308A7000230A200A3018A0180218316B7
:100A2000DF0083128A01B9217D308316E002831230
:100A30008A01B9218A113F2D8A01B921903083168C
:100A40005F078312B200FF300318013EB300320883
:100A5000A6003308A7000230A200A3018A0180216A
:100A6000B2002508B30032038316DF0083128A0127
:100A7000B9211F308316E00283128A01B9218A014D
:100A8000B9218316DE0A83128A01B9218A11DC2575
:100A90008A01B92183160030E91A01308312B200AD
:100AA000B3010130A600A7013208A2003308A30059
:100AB0008A018021B2002508B30083160030691B2B
:100AC00001308312B400B5010230A600A70134083A
:100AD000A2003508A3008A018021B4002508B500D2
:100AE0003208B40733080318013EB50783160030F7
:100AF000E91B01308312B600B7010430A600A7013C
:100B00003608A2003708A3008A018021B600250814
:100B1000B700340836078316E10083128A01B92131
:100B2000640083166108023C8A158312031949295F
:100B30008A01B921640083166108033C8A15831277
:100B4000031997298A01B921640083166108043CBE
:100B50008A1583120319DB298A01B92164008316DF
:100B60006108053C8A15831203191F2A8A01B921DD
:100B7000640083166108063C8A1583120319682AEB
:100B80008A01B921640083166108073C8A15831223
:100B90000319B12A8A01B92120308A011720CC30EB
:100BA0008A011720D2308A011720B2308A0117201B
:100BB0008A01B9218A159F2C8A01B9210130831637
:100BC00060058312B200B301320C83160318E814D7
:100BD000031CE81083128A01B921023083166005D4
:100BE0008312B200B3010310B30CB20C320C8316A3
:100BF00003186815031C681183128A01B921043097
:100C0000831660058312B200B3013208A0003308D6
:100C1000A10002308A014321B2002108B300320C46
:100C200083160318E815031CE81183128A01B92101
:100C30000830831660058312B200B3013208A000A9
:100C40003308A10003308A014321B2002108B30018
:100C5000320C831603186816031C681283128A016B
:100C6000B9211030831660058312B200B301320837
:100C7000A0003308A10004308A014321B2002108FA
:100C8000B300320C83160318E816031CE812831213
:100C90008A01B9212030831660058312B200B301A6
:100CA0003208A0003308A10005308A014321B200B8
:100CB0002108B300320C831603186817031C68134D
:100CC00083128A01B9214030831660058312B20075
:100CD000B3013208A0003308A10006308A01432185
:100CE000B2002108B300320C83160318E817031C66
:100CF000E81383128A01B9218030831660058312BC
:100D0000B200B3013208A0003308A10007308A0105
:100D10004321B2002108B300320C83160318691472
:100D2000031C691083128A01B921013083165F0503
:100D30008312B200B301320C83160318E914031CAA
:100D4000E91083128A01B921023083165F058312EC
:100D5000B200B3010310B30CB20C320C83160318AB
:100D60006915031C691183128A01B92104308316A5
:100D70005F058312B200B3013208A0003308A1005E
:100D800002308A014321B2002108B300320C8316DD
:100D90000318E915031CE91183128A01B9210830EF
:100DA00083165F058312B200B3013208A000330836
:100DB000A10003308A014321B2002108B300320CA4
:100DC000831603186916031C691283128A01B9215C
:100DD000103083165F058312B200B3013208A00001
:100DE0003308A10004308A014321B2002108B30076
:100DF000320C83160318E916031CE91283128A01C8
:100E0000B921203083165F058312B200B301320886
:100E1000A0003308A10005308A014321B200210857
:100E2000B300320C831603186917031C691383126D
:100E30008A01B921403083165F058312B200B301E5
:100E40003208A0003308A10006308A014321B20015
:100E50002108B300320C83160318E917031CE913A9
:100E600083128A01B921803083165F058312B20094
:100E7000B3013208A0003308A10007308A014321E2
:100E8000B2002108B300320C831603186A14031C45
:100E90006A1083128A01B92183160130E600831299
:100EA00064000930831666028A11831203186D2FBD
:100EB0008A01B921EB30840083166608003E831254
:100EC0008A01052003108A0110208A01B9218316A6
:100ED000E60A8A118312031D502F8A01B921831655
:100EE0000030E81801308312B200B301320C8316CF
:100EF0000318EA14031CEA1083128A01B92183162D
:100F00000030681901308312B200B301320C83162D
:100F100003186A15031C6A1183128A01B92183160A
:100F20000030E81901308312B200B301320C83168D
:100F30000318EA15031CEA1183128A01B9218316EA
:100F40000030681A01308312B200B301320C8316EC
:100F500003186A16031C6A1283128A01B9218316C8
:100F60000030E81A01308312B200B301320C83164C
:100F70000318EA16031CEA1283128A01B9218316A8
:100F80000030681B01308312B200B301320C8316AB
:100F900003186A17031C6A1383128A01B921831686
:100FA0000030E81B01308312B200B301320C83160B
:100FB0000318EA17031CEA1383128A01B921831666
:100FC0000030E91801308312B200B301320C8316ED
:100FD00003186B14031C6B1083128A01B9210800DB
:100FE0008A01B9218A1588268A01B9218316E6016A
:100FF00083128A01B921640083166008DE3C8A15D9
:101000008312031D1A288A01B92183160130E600D4
:1010100083128A01B9218316DE0A83128A01B9215B
:101020008316DE30E30083128A01B9218A158826EF
:101030008A01B9218A01B921640083166008DF3C66
:101040008A158312031D3B288A01B92183160230B9
:10105000E60083128A01B9218316DE0A83128A010F
:10106000B9218316DF30E30083128A01B9218A1582
:1010700088268A01B9218A01B921A03083165F022E
:10108000E50083128A01B9218316650883128A015B
:101090001E218316E00083128A01B92183162530B0
:1010A000DF0083128A01B921640083166508103CB1
:1010B0008A158312031D602883162130DF008312F6
:1010C0008A01B92164000630831665028A158312ED
:1010D00003186E2883162130DF0083128A01B9219C
:1010E00083166608E00783128A01B92108008A0185
:1010F000B9218A1588268A01B92183160030691B17
:1011000001308312B200B30183160030E91B0130B5
:101110008312B400B5013408A6003508A7000230D8
:10112000A200A3018A018021B4002508B50032087D
:1011300034078316E10083128A01B9216400831603
:101140006108013C8A158312031DAA2883166913BE
:10115000E91383128A01B921640083166108023CF5
:101160008A158312031DB82883166917E9138312A1
:101170008A01B921640083166108033C8A15831231
:10118000031DC62883166913E91783128A01B92142
:1011900083160030E91801308312B200B301320C1B
:1011A00083160318EA14031CEA1083128A01B9217A
:1011B00083160030691901308312B200B301320C7A
:1011C000831603186A15031C6A1183128A01B92158
:1011D00083160030E91901308312B200B301320CDA
:1011E00083160318EA15031CEA1183128A01B92138
:1011F00083160030691A01308312B200B301320C39
:10120000831603186A16031C6A1283128A01B92115
:1012100083160030E91A01308312B200B301320C98
:1012200083160318EA16031CEA1283128A01B921F5
:1012300083166A1383128A01B9218316EA13831273
:101240008A01B92183160030691B01308312B20074
:10125000B301320C831603186B14031C6B1083123A
:101260008A01B92183160030E91B01308312B200D4
:10127000B301320C83160318EB14031CEB1083121A
:101280008A01B9218316EB1783128A01B9218A15C5
:10129000042B8A01B92183166A1383128A01B921AA
:1012A0008316EA1383128A01B92183160030691963
:1012B00001308312B200B301320C83160318EB1411
:1012C000031CEB1083128A01B92183160030E9193F
:1012D00001308312B200B301320C831603186B1570
:1012E000031C6B1183128A01B92183160030681B1D
:1012F00001308312B200B301320C83160318EB15D0
:10130000031CEB1183128A01B92183160030E81BFC
:1013100001308312B200B301320C831603186B162E
:10132000031C6B1283128A01B9218A15042B8A01CE
:10133000B92183160030691901308312B200B3015C
:10134000320C83160318EB14031CEB1083128A0172
:10135000B92183160030E91901308312B200B301BC
:10136000320C831603186B15031C6B1183128A0150
:10137000B92183160030691A01308312B200B3011B
:10138000320C83160318EB15031CEB1183128A0130
:10139000B92183160030E91B01308312B200B3017A
:1013A000320C831603186B16031C6B1283128A010E
:1013B000B9218A15042B8A01B921831600306919D5
:1013C00001308312B200B301320C83160318EB1400
:1013D000031CEB1083128A01B92183160030E9192E
:1013E00001308312B200B301320C831603186B155F
:1013F000031C6B1183128A01B92183160030691A0C
:1014000001308312B200B301320C83160318EB15BE
:10141000031CEB1183128A01B92183160030E91BEA
:1014200001308312B200B301320C831603186B161D
:10143000031C6B1283128A01B9218A15042B8A01BD
:10144000B92183160030691901308312B200B3014B
:10145000320C83160318EB14031CEB1083128A0161
:10146000B92183160030E91901308312B200B301AB
:10147000320C831603186B15031C6B1183128A013F
:10148000B92183160030691A01308312B200B3010A
:10149000320C83160318EB15031CEB1183128A011F
:1014A000B92183160030691B01308312B200B301E9
:1014B000320C831603186B16031C6B1283128A01FD
:1014C000B9218316EB1683128A01B9218A15042BE0
:1014D0008A01B92183160030691901308312B200E4
:1014E000B301320C83160318EB14031CEB108312A8
:1014F0008A01B92183160030E91901308312B20044
:10150000B301320C831603186B15031C6B11831285
:101510008A01B92183160030691A01308312B200A2
:10152000B301320C83160318EB15031CEB11831265
:101530008A01B92183160030691B01308312B20081
:10154000B301320C831603186B16031C6B12831243
:101550008A01B9218316EB1683128A01B9218A15F3
:10156000042B8A01B92183166A1383128A01B921D7
:101570008316EA1383128A01B92183160030691990
:1015800001308312B200B301320C83160318EB143E
:10159000031CEB1083128A01B92183160030E9196C
:1015A00001308312B200B301320C831603186B159D
:1015B000031C6B1183128A01B92183160030681B4A
:1015C00001308312B200B301320C83160318EB15FD
:1015D000031CEB1183128A01B92183160030E81B2A
:1015E00001308312B200B301320C831603186B165C
:1015F000031C6B1283128A01B9218316EB16831226
:101600008A01B9218A15042B8A01B9218316003079
:10161000EA1801308312B200B3010130A600A7011D
:101620003208A2003308A3008A018021B2002508F5
:10163000B300831600306A1901308312B400B5017B
:101640000230A600A7013408A2003508A3008A01D1
:101650008021B4002508B5003208B4073308031808
:10166000013EB50783160030EA1901308312B60037
:10167000B7010430A600A7013608A2003708A3006E
:101680008A018021B6002508B7003408B60735085E
:101690000318013EB707831600306A1A013083121F
:1016A000B800B9010830A600A7013808A20039081F
:1016B000A3008A018021B8002508B9003608B807C0
:1016C00037080318013EB90783160030EA1A0130C3
:1016D0008312BA00BB011030A600A7013A08A2008D
:1016E0003B08A3008A018021BA002508BB00380806
:1016F000BA0739080318013EBB07831600306A1B7E
:1017000001308312BC00BD012030A600A7013C08B7
:10171000A2003D08A3008A018021BC002508BD006D
:101720003A08BC073B080318013EBD07831600308A
:10173000EA1B01308312BE00BF014030A600A701A2
:101740003E08A2003F08A3008A018021BE002508B0
:10175000BF003C08BE073D080318013EBF078316C3
:1017600000306B1801308312C000C1018030A60028
:10177000A7014008A2004108A3008A018021C000FF
:101780002508C1003E08C0073F080318013EC107F5
:1017900083166408BE3E84008312400880008A01DC
:1017A000B92183160030EB1801308312B200B30167
:1017B0000130A600A7013208A2003308A3008A0165
:1017C0008021B2002508B300831600306B19013068
:1017D0008312B400B5010230A600A7013408A200AC
:1017E0003508A3008A018021B4002508B50032081D
:1017F000B40733080318013EB50783160030EB1910
:1018000001308312B600B7010430A600A7013608E4
:10181000A2003708A3008A018021B6002508B7007E
:101820003408B60735080318013EB70783160030A1
:101830006B1A01308312B800B9010830A600A70165
:101840003808A2003908A3008A018021B8002508C1
:10185000B9003608B80737080318013EB9078316E0
:101860000030EB1A01308312BA00BB011030A60021
:10187000A7013A08A2003B08A3008A018021BA0010
:101880002508BB003808BA0739080318013EBB0712
:10189000831600306B1B01308312BC00BD01203069
:1018A000A600A7013C08A2003D08A3008A018021F0
:1018B000BC002508BD003A08BC073B080318013EE0
:1018C000BD0783160030EB1B01308312BE00BF0141
:1018D0004030A600A7013E08A2003F08A3008A01ED
:1018E0008021BE002508BF003C08BE073D08031844
:1018F000013EBF07831600306C1801308312C00010
:10190000C1018030A600A7014008A2004108A30041
:101910008A018021C0002508C1003E08C0073F0899
:101920000318013EC10783166408A03E8400831299
:10193000400880008A01B9218316E40A83128A01D3
:10194000B9218316DE0A8A118312031D132C8A0122
:10195000B92108008A01B9218316DD0183128A01A9
:10196000B921FB01FC018A01B921FD018A01B921DC
:101970007D088316EE0083128A01B9218A15FC25A1
:101980008A01B92183165D08EE0083128A01B9210C
:101990008A15FC258A01B92183165E08EE008312A0
:1019A0008A01B9218A15FC258A01B9218316EE0125
:1019B00083128A01B9218A15FC258A01B9218A1569
:1019C0001C268A01B921FF308A0123218A01B9210D
:1019D00008008A01B9218316DD0183128A01B92129
:1019E000FB01FC018A01B9217D088316EE008312F8
:1019F0008A01B9218A15FC258A01B9218316EE01D5
:101A000083128A01B9218A15FC258A01B92183161E
:101A10005C08EE0083128A01B9218A15FC258A012F
:101A2000B92183160130EE0083128A01B9218A158B
:101A3000FC258A01B9218A151C268A01B921FB01DE
:101A4000FC018A01B9218316EE0183128A01B921B2
:101A50008A15FC258A01B92183165D08EE008312E0
:101A60008A01B9218A15FC258A01B9218316EE0164
:101A700083128A01B9218A15FC258A01B9218316AE
:101A8000EE0183128A01B9218A15FC258A01B92148
:101A900083168B30EE0083128A01B9218A15FC254A
:101AA0008A01B9218316DE01831264000B3083168C
:101AB0005E028A1583120318772D8A01B9218316D5
:101AC000EE0183128A01B9218A15FC258A01B92108
:101AD0008316EE0183128A01B9218A15FC258A0139
:101AE000B9218316DE0A8A158312031D552D8A013A
:101AF000B9218316DE01831264001E3083165E0254
:101B00008A1583120318A62D8A01B92183165E084F
:101B1000BE3E84000008EE0083128A01B9218A15B6
:101B2000FC258A01B92183165E08A03E84000008C6
:101B3000EE0083128A01B9218A15FC258A01B92198
:101B40008316DE0A8A158312031D7C2D8A01B921B2
:101B50008316FF30EE0083128A01B9218316DE015D
:101B600083126400AC3083165E028A158312031858
:101B7000C52D8A01B9218A15FC258A01B921831650
:101B8000DE0A8A158312031DB12D8A01B9218A1537
:101B90001C268A01B9218316DE01831264001E30DF
:101BA00083165E028A1583120318F92D8A01B92162
:101BB00083165E08483E84000030800083128A014C
:101BC000B92183165E08BE3E840000308000831277
:101BD0008A01B92183165E08A03E8400003080008F
:101BE00083128A01B9218316DE0A8A158312031D26
:101BF000CE2D8A01B92108008A01B9210630C6001C
:101C00000430C4002030AA004030AB00AE01AF0168
:101C100083166E0883128A01CE208A01B9218A15A3
:101C200078268A01B92183166E088312FB070318F0
:101C3000FC0A8A01B92108008A01B921FF307B051D
:101C4000FF008A01B92100307B05B200FF307C051E
:101C5000B3003208A0003308A100A2010130A300A4
:101C60008A016421FE008A01B9210630C6000430D1
:101C7000C4002030AA004030AB00AE01AF017E08A6
:101C80008A01CE208A01B9218A1578268A01B921D4
:101C90000630C6000430C4002030AA004030AB003B
:101CA000AE01AF017F088A01CE208A01B9218A15D1
:101CB00078268A01B9210630C6000430C4002030DD
:101CC000AA004030AB00AE01AF01EF308A01CE2058
:101CD0008A01B9218A1578268A01B9218316DD0A7D
:101CE00083128A01B9218A1580268A01B921080048
:101CF0008A01B9210A308A0130218A01B9210800FC
:101D00008A01B92164308A0123218A01B92108009E
:101D10008A01B9218316630883128A0117208A0178
:101D2000B9216400831662080F3C8A158312031DD3
:101D30009F2EFE308A011720C0308A0117208A01A9
:101D4000B9218316E20A83128A01B92108006400CE
:101D50008A150B1DAE2E83166C1483120B1109000D
:101D6000FF3FFF3FFF3FFF3FFF3FFF3FFF3FFF3F83
:101D7000FF3FFF3FFF3FFF3FFF3FFF3FFF3FFF3F73
:101D8000FF3FFF3FFF3FFF3FFF3FFF3FFF3FFF3F63
:101D9000FF3FFF3FFF3FFF3FFF3FFF3FFF3FFF3F53
:1042000020002300560057002200260072002100E3
:104210002300250027002900630065006700430094
:104220003C0022002400260028002A002B002D003C
:104230002F00310033003500370039003B003D00CE
:104240003F0041004400460048004A004B004C003B
:104250004D004E004F005200550058005B005E00BC
:104260005F00600061006200640066006800690031
:104270006A006B006C006D006F007300200020006E
:10428000FF00FF00FF00FF00FF00FF00FF00FF0036
:10429000FF00FF00FF00FF00FF00FF00FF00FF0026
:1042A000FF00FF00FF00FF00FF00FF00FF00FF0016
:1042B000FF00FF00FF00FF00FF00FF00FF00FF0006
:1042C000FF00FF00FF00FF00FF00FF00FF00FF00F6
:1042D000FF00FF00FF00FF00FF00FF00FF00FF00E6
:1042E000FF00FF00FF00FF00FF00FF00FF00FF00D6
:1042F000FF00FF00FF00FF00FF00FF00FF00FF00C6
:10430000FF00FF00FF00FF00FF00FF00FF00FF00B5
:10431000FF00FF00FF00FF00FF00FF00FF00FF00A5
:10432000FF00FF00FF00FF00FF00FF00FF00FF0095
:10433000FF00FF00FF00FF00FF00FF00FF00FF0085
:10434000FF00FF00FF00FF00FF00FF00FF00FF0075
:10435000FF00FF00FF00FF00FF00FF00FF00FF0065
:10436000FF00FF00FF00FF00FF00FF00FF00FF0055
:10437000FF00FF00FF00FF00FF00FF00FF00FF0045
:10438000FF00FF00FF00FF00FF00FF00FF00FF0035
:10439000FF00FF00FF00FF00FF00FF00FF00FF0025
:1043A000FF00FF00FF00FF00FF00FF00FF00FF0015
:1043B000FF00FF00FF00FF00FF00FF00FF00FF0005
:1043C000FF00FF00FF00FF00FF00FF00FF00FF00F5
:1043D000FF00FF00FF00FF00FF00FF00FF00FF00E5
:1043E000FF00FF00FF00FF00FF00FF00FF00FF00D5
:1043F000FF00FF00FF00FF00FF00FF00FF00FF00C5
:1080000020002300560057002200260072002100A5
:108010002300250027002900630065006700430056
:108020003C0022002400260028002A002B002D00FE
:108030002F00310033003500370039003B003D0090
:108040003F0041004400460048004A004B004C00FD
:108050004D004E004F005200550058005B005E007E
:108060005F006000610062006400660068006900F3
:108070006A006B006C006D006F0073002000200030
:10808000FF00FF00FF00FF00FF00FF00FF00FF00F8
:10809000FF00FF00FF00FF00FF00FF00FF00FF00E8
:1080A000FF00FF00FF00FF00FF00FF00FF00FF00D8
:1080B000FF00FF00FF00FF00FF00FF00FF00FF00C8
:1080C000FF00FF00FF00FF00FF00FF00FF00FF00B8
:1080D000FF00FF00FF00FF00FF00FF00FF00FF00A8
:1080E000FF00FF00FF00FF00FF00FF00FF00FF0098
:1080F000FF00FF00FF00FF00FF00FF00FF00FF0088
:10810000FF00FF00FF00FF00FF00FF00FF00FF0077
:10811000FF00FF00FF00FF00FF00FF00FF00FF0067
:10812000FF00FF00FF00FF00FF00FF00FF00FF0057
:10813000FF00FF00FF00FF00FF00FF00FF00FF0047
:10814000FF00FF00FF00FF00FF00FF00FF00FF0037
:10815000FF00FF00FF00FF00FF00FF00FF00FF0027
:10816000FF00FF00FF00FF00FF00FF00FF00FF0017
:10817000FF00FF00FF00FF00FF00FF00FF00FF0007
:10818000FF00FF00FF00FF00FF00FF00FF00FF00F7
:10819000FF00FF00FF00FF00FF00FF00FF00FF00E7
:1081A000FF00FF00FF00FF00FF00FF00FF00FF00D7
:1081B000FF00FF00FF00FF00FF00FF00FF00FF00C7
:1081C000FF00FF00FF00FF00FF00FF00FF00FF00B7
:1081D000FF00FF00FF00FF00FF00FF00FF00FF00A7
:1081E000FF00FF00FF00FF00FF00FF00FF00FF0097
:1081F000FF00FF00FF00FF00FF00FF00FF00FF0087
:08400000FF3FFF3FFF3FFF3FC0
:02400E00463F2B
:10401000FF3FFF3FFF3FFF3FFF3FFF3FFF3FFF3FB0
:00000001FF
